:020000040000FA
:100000008B018A018301AB28F000030E8301F1000C
:100010000408F2008C1E4C28981C18194928181C3A
:1000200028283711B6011A08B100B7196328603AB9
:10003000031925283108320603194128A03A03196B
:100040002528603A03193C286328B5013715632831
:100050002030360784001A08371D63288000B50653
:10006000B60A20080F39023E3606031D63283711F1
:10007000B5080319B71563280614203099009900B4
:100080005A28371C6328061483160C168312B714DB
:1000900050281A08181218160C1E6328B71C5A2864
:1000A000A0303307840000089900B30AB40B63281A
:1000B0003710B7108316981C5B280C128312602827
:1000C00061286228061072088400710E8300F00E09
:1000D000700E090082073F3406345B344F346634B7
:1000E0006D347D3407347F346F343F0E0739820717
:1000F0000134023404340834103420344034803461
:10010000BD19CF01CF08031908000301CF1A013030
:100110004F1B0230CF180330CF0151078207EC2A62
:10012000342B012B472B0A2BF32AFC2A472B382B85
:10013000162B3C2B472B0800612B6D2BAB28612B1A
:100140004C2B592BAB28612B7B2B762BAB281A2BF6
:10015000062B042B472B9801850186018316F63068
:100160008600FF30850020308C00813081000B300C
:100170008E0000309F00831205309F0020308400E5
:100180008001840A841FC028922245222224A023B1
:10019000C0308B004030C900CA0056224D182D29AE
:1001A00001303524BF006030C100ED21EA2022215A
:1001B0000C1827213718D728F221EA203823DA2211
:1001C00004223C1622210C1CE228F0202221AB2321
:1001D0008020E628313090008E018F010C1008003D
:1001E00090010C1008000C1CFC28F020D108031D05
:1001F000FC283F08B222C8228C1C08008C109F1FCC
:100200000629C7304306031DC30A0929C308031D75
:10021000C303430C8400040C3F399500430E30396E
:100220000C3897004308C5070318C60AC40F080016
:100230004608C800C501C6013C170310CC0D0318C1
:100240004C140800F3205A22B719332108000C106F
:10025000F930C9000730CA00080063231124F320D5
:100260005A2280202E292008613A031D6329210883
:10027000031D4529BD18EB29BD11BD143D10F930F2
:10028000C9003F30CA00C822E929013A031D552997
:10029000BD11BD103D103F08B222C8223D080B39E8
:1002A0000319E929B7110422E929033A031DEB29AF
:1002B000BD19EB29BD15BD103D106D30C90073305F
:1002C000CA00C822E929033A031D73292108223AEA
:1002D000031DEB292208BD00BD195D29BD183F296A
:1002E0003D188B294B29013A031D7F292108213A0A
:1002F000031DEB292208B8002308B900EB292008C8
:10030000813A031D91292108031DEB293D18EB2992
:10031000BD11BD103D14F930C9006D30CA00C822AE
:10032000E9292008E13A031DA0292108883A031D84
:10033000EB296D30C9004030CA00CC30CC00EB292D
:10034000033A031DAD292108F039203A031DEB299A
:100350003C153F08BE00C101CD29013A031DC0294B
:100360002108403A031DEB2922083F39031DEB29E0
:1003700023083F06031DEB293C14C8223C16EB2939
:10038000073A031DDD292108F039031DEB293C1133
:100390003F08BE0023081F39C100A21BC116211C43
:1003A000A11841172119C11722087F39C0003C103C
:1003B000A1193C14C8223C16EB29013A031DEB2974
:1003C0002108F039103A031DEB293C152508BE0021
:1003D000CA29D101C822B7110800213030222130AA
:1003E0003822412A2130302224303822412A8030DC
:1003F0003022412A2130302280303822412A2130D7
:10040000302281303822412AE33030220030382235
:10041000003038223F083822412AE43030221030A0
:10042000411B1230C11B13303822003038223F08E4
:1004300038224008C11A803838223C10C8223F08B0
:10044000F30001303E24412AE430302220303822AB
:10045000003038223F08382241081F3938221D2A2F
:10046000BA00B71933213718312AB301B4013A0859
:10047000BB00A030340784003B088000B306B40AF8
:1004800008003308382237140800003035241F399B
:10049000031901304038B2008400040E8406040CB5
:1004A00084060419840A0418B21708004B08851A38
:1004B000CD0408000B1D08000B1156228316D930FD
:1004C0008504F030860483129222CC1B08004B086E
:1004D0000319712A4A050319712A8316051283121A
:1004E0000512CB1B7D2A4B080319803049050319DF
:1004F0007D2A83168511831285114B1C08004E0935
:100500004D05CF000319862A3730D0004D08CE00A4
:10051000CD014E0803190800D00B0800CF0016309B
:10052000D00008004B08003CCB0DFF30CB0803196E
:10053000103A4B18013ACB1A803A4B1B403ACB1B6E
:10054000083A831685058312FF3A85044B0D840013
:10055000840D040DF039FF3A831686058312FF3AA5
:1005600086040800CA0064304A020318C42AC9017C
:100570000A30C90ACA020318B92A4A076A20CA00FF
:1005800049036A20C90008003830CA005C30C22A1A
:100590000301D108031D01303C18CC30BD18C33015
:1005A0003D18C330BD19C330CC0008003F080F39D7
:1005B000043E0800BC12D6223524F30075207305D2
:1005C000031DBC160800D6223524F3007520F30461
:1005D000BC1EF3063B2463343830C900CA01043022
:1005E000D100C8220800E3223F060319BF01BF0A59
:1005F000DA2204223F08B22AE322BF030319BF0014
:10060000F82A1030C106242A0230082B0130082BAA
:10061000C10624220830C1180130CA000830411830
:100620000130C9001830D100C82208002030C106AE
:10063000BC060D22C208031D382BC11E282B5E30BC
:10064000C9000830411B4030C11B0130CA00302BAB
:100650000830411B4030C11B0130C9005E30CA0068
:100660000830D100C82208002030C106BC060D2287
:10067000D101C8223F08B22AC208031D08008030F9
:10068000C11F4030411BC030C1060D221A2B3D183E
:10069000FF29BD18482BFA2900303524F300F30A4E
:1006A0002030730601300319F30000303E24730834
:1006B000B22A00303524F300F3031F300319F3008E
:1006C000552BBC1D662BBC117730682BBC157330C5
:1006D000C900CA010C30D10008001430BC1D103014
:1006E000D100BC19080000303524B22A4808C700E0
:1006F000F30002303E2C831612088312F500F40139
:1007000008308400882B0310F40DF50D03188C2B92
:1007100048087502031C8F2B4808F5027414840BDB
:10072000832B74089623F30003303E2C8400841F2F
:10073000041B3130841E313083169200831208006E
:100740000330352496233C3092000C309700023061
:100750003524C70008003C1F08003C133718080068
:10076000B71247080319C02B48020318B92B003CE5
:10077000B716FC3E031C030184000310840DC22B3A
:10078000480884003C1AFF2B411BD62BC11BE62BCB
:100790000310840C0310840C0310840C0E3001240D
:1007A000031908000724031D013EF52B0310840CD8
:1007B0000310840C1C300124031908000724031DB6
:1007C000033E8400040C03181038F52B7E300124FE
:1007D00003190800C2060310420C0924031D013E40
:1007E000D108031DF52B4218CA17C000C20803190F
:1007F0000D2A3C08370641062039C1060D2A3C1255
:1008000008000402031884020408420608000408D1
:10081000C200D108031D0F2CB222CC01EA204208ED
:1008200008003C1F08003C135108143A031D08003F
:100830000310480CB2224818CA1748084706031983
:10084000C91708000610B701B601831603309900D6
:10085000643098008312D03098000301FF3E031DDE
:100860002E2C1A081A081A08080083169B001C145C
:100870001A0883120800831637243F2C3524730688
:1008800003190800730883169A001C158B13553042
:100890009D00AA309D009C148B171C119C184E2C97
:0408A00083120800B7
:02400E00503F21
:104200000100030000003100000000000000000079
:10421000000000000000000000000000000000009E
:104220000000000000000000530069006D007000F5
:104230006C00650020004D006100750073002000D7
:1042400076002E0034000A0046002E004300610074
:10425000C300B1006100640061002D003E004A000F
:104260002E0046007500C4008D0069006B002D0013
:104270003E0048002E0048006100660074006D009A
:1042800061006E006E000A00310039002F0030001E
:0842900032002F003000350060
:00000001FF
